:100000008316043085000030860083129C009F1305
:10001000AE2882070334073406340434023406342D
:100020000734033405340234023403340534043411
:1000300002340734063407340434033402340534FC
:1000400007340634033402340234033404340534F0
:1000500004340334073404340634073402340334DC
:1000600004340534013400309100083092001C3013
:10007000930008309400003095007C2803309100F4
:10008000033092000030930060309400603095009F
:100090007C28033091000B3092001C3093006830B4
:1000A0009400603095007C286330910063309200AA
:1000B0000030930063309400633095007C286330F7
:1000C00091006B3092001C3093006B3094006330D1
:1000D00095007C289F1F7728EB309100803093009B
:1000E0006B3092006B3094006B3095007C286B3045
:1000F00091000030930070288514000085101108CD
:1001000086008F20120886008F20130886008F201B
:10011000140886008F20150886008F2008009B0B8E
:100120008F280030860005140000051008001C0808
:1001300009209D009D0B9F2800309C0097289D0B57
:10014000A22833289D0BA5283E289D0BA8284928C6
:100150009D0BAB2854289D0B6A285F2830308C00FB
:1001600097208C0BB0289C0A40308C0097208C0B79
:10017000B6289C0A50308C0097208C0BBC289C0A17
:1001800060308C0097208C0BC2289C0A70308C0049
:1001900097208C0BC8289C0A9F179720051DCC28F8
:0401A0009F13AE28D3
:00000001FF
